:020000040000FA
:1000000064008B0185018316803081001F308500DC
:100010008601831286017220FF30860072208901DA
:100020008316081483120808F0398E006400083023
:100030008C000E04860000000508031D37280430DC
:100040008C000E04860000000508031D37280230CE
:100050008C000E04860000000508031D37280130BF
:100060008C000E04860000000508031916288D0078
:100070000D0E0C048F008E010E0850200F02031984
:1000800045288E0A0E1E3C2848288E0E0E08612038
:1000900064000F300E0486000508031D482816284A
:1000A00082078834223444341234483441342434AE
:1000B0001134283418348234813484341434423472
:1000C00021346400890188008316081555308900A1
:1000D000AA3089008814881C6F2864006B280811D6
:0E00E0008312080090016400900B7328080042
:02400E00FD3F74
:00000001FF
